:020000040020DA
:100000002C75002055F8210085F8210089F8210081
:100010008DF821008DF821008DF8210000000000EE
:100020000000000000000000000000008DF821002A
:100030008DF82100000000008DF821005DF5210001
:100040008DF821008DF821008DF821008DF8210018
:10005000000000008DF821008DF821008DF82100AE
:100060008DF82100000000000000000000000000EA
:1000700000000000000000008DF8210000000000DA
:1000800000000000000000008DF821008DF8210024
:100090008DF821008DF821008DF821008DF82100C8
:1000A0008DF821008DF82100B94A20001F4B200057
:1000B0008DF821008DF821008DF821008DF82100A8
:1000C0005DF92100754A20008DF821008DF821008E
:1000D0008DF821000000000000000000000000007A
:1000E0000000000000000000000000000000000010
:1000F0008DF82100000000008DF8210000000000B4
:1001000010B5DFF8B80B0FF2B961C84C41650FF2BA
:10011000F97181650FF27551E1620FF2355121637A
:100120000FF6290161630FF65501A1630FF2F97112
:10013000E1630FF2C13121640FF2B55141640FF256
:100140000D6181640FF27551C1640FF6A90101655B
:10015000206908B102F08EFBDFF8B40B0B49A060F8
:100160000B22082020730020206181F820002075D8
:10017000002104F1150002F0C7FB04F12000BDE8E6
:1001800010400B22002102F0BFBB0000C44200203F
:100190003EB504460520E082032020756068401EBD
:1001A0006060411E616094F83A10017094F83A0062
:1001B00010B14FF6FF7121876068411E6160218F89
:1001C000090A01706168208F087004F12F01207AFC
:1001D000C01C2072684602F0D0FDDFF8F809C38C1D
:1001E00003228DF8082003216A46204601F0DEFC38
:1001F000050004BF204600F0B2FE28463EBD70B5A3
:100200000D46044661680498160A01F8016D01F86C
:10021000020C01F8012CDFF8BC09428D120A01F82A
:10022000032C408D01F8040C180A01F8050C01F8A4
:10023000063D227A606861608218521A2272287A1A
:10024000DFF82C1C03280CBF01200020E0820B22C9
:100250000920207504F1240002F03EFB4FF6FF73E5
:100260002A460321204601F0A1FC050004BF2046D8
:1002700000F075FE284670BDDFF8F81B897A082962
:1002800081B0A8BF072101700078C006000E01B040
:10029000704700002DE9F04706460F46904602F0F1
:1002A00073FD0025DFF8CC9BD9F80040B0F1010ABE
:1002B0006AEB0A0A4FEADA7A09E0F61F411D304676
:1002C00002F05BFD54F8084C761E10357F1EF8B224
:1002D00068B10AE0607E410605D560684178C1F3E7
:1002E00081010329E9D054F8084C002CF2D1BAF16D
:1002F000000F18BF02F044FD02F046FD421E92417D
:10030000D9F80000D20F2C46E8B143685D78C5F3F8
:100310008105022D14D1457E690609D59B7906F821
:100320000139641C43685D7906F801597F1E07E0B6
:10033000037E9D0604D5012588F80050FBB213B159
:1003400050F8080CE0E70AB102F01AFD3470701E94
:10035000BDE8F0872DE9F84384B00D4600218046C2
:100360008DF8001091460DF10100FFF785FFDFF8D1
:1003700064783E7B86194136F6B2304602F0F4FAD4
:1003800004004ED0A0196060002020723A7B6068A3
:10039000114649424618B968304602F09DFA9DF868
:1003A00001106A46701EFFF775FF00217E4A01703A
:1003B000137879789B0143EAC11343EA091343F0A8
:1003C0000F0300F8013C48EA051100F8021D227AEB
:1003D000616860608A18121A00202272E08220751B
:1003E0008DF80C000B22DFF8E81B04F1240002F06A
:1003F00073FA9DF8000018B1E18A41F00801E1822A
:100400004FF6FE71788D8842ACBF03210221002394
:1004100001AA204601F0CAFB0028204602D002F0C3
:10042000B5FA002005B0BDE8F08300008850002038
:10043000F8B5074602F0A8FC461EDFF8380A046843
:10044000B641F60F00250EE0617E080609D57968F1
:10045000606801F057FB20B1607E00F0BF0060765D
:10046000254654F8084C002CEED11DB1687E40F0B2
:10047000400068761EB1BDE8F14002F081BCF1BDDC
:100480002DE9F8438046894602F07EFC0026471E8F
:10049000DFF8E0090568BF41FF0F00240AE02C46A1
:1004A000617E207E41F0100140F080006176207670
:1004B00055F8085C9DB1687E0106F9D56A68494621
:1004C000404601F03BFB0028F2D0002CE7D0207D15
:1004D000012804D16068017841F0100101700FB16A
:1004E00002F04EFC14B100F0C7FC01263046BDE816
:1004F000F28300002DE9FC410025009502F044FC48
:1005000000F04BF80EE054F8088C2A462146384695
:1005100002F006FB2146684602F0BEFAB87A411E98
:100520004446B972CCB1607E010605D5608A401E92
:10053000608280B20028E6D0254654F8084CF1E7E6
:10054000FFF776FF607E410759BFF0206070E92118
:100550006170204600F0E3FB18E00EB102F010FCE1
:10056000B87A98B1DFF86C16487B0F281EBFDFF809
:10057000281B91F82000002808D1DFF83C4C2046C9
:1005800002F0B5F83021204602F098F8684602F0F3
:100590009EFA0400D4D1BDE8F381DFF8007B3C680B
:1005A000461EB641F60F7047F44F002070B5054661
:1005B000FFF73EFFDFF8BC48DFF81866A06C804705
:1005C0000128F08D08BF401C6882A07A002804BF73
:1005D000717B0F2908D1DFF8E05B284602F087F82D
:1005E0003021284602F06AF802F0CEFBA17A00F032
:1005F0002AF8A17218B1BDE8704002F0C1BB70BD0D
:1006000038B50446DFF86C58607E00F0EF00607685
:100610002046FFF70DFF2146284602F070FA02F04F
:10062000B3FBA97A00F00FF8A97208B102F0A8FB99
:10063000DFF8A005417B0F2904D1BDE83240082036
:1006400001F0A8B831BD401E8041491CC00F704761
:1006500010B5DFF880150446487886B0A0B10121B6
:1006600000208DF800108DF8010000F03AF8616864
:1006700008788DF80A0004F10F010DF10B0001F06C
:10068000EBFB684602F0A4FC06B010BD10B50446B2
:10069000FFF77EFDDC2818BFDD2808D0E42818BF4E
:1006A000F32804D0DE281CBFDF28DB2805D1014653
:1006B0002046BDE8104001F073B810BD10B586B0FB
:1006C000044606208DF8000000F00BF804F10F013D
:1006D0000DF10A0001F0C0FB684602F079FC06B09B
:1006E00010BD04F11C010DF1020002F046BB000038
:1006F00038B5044604F1380584B0A87820B304F175
:100700002F0101A802F039FB6248017D03880091A6
:1007100003228DF80C2001A92A882046FFF76FFDDF
:100720000146DC2918BFDD290BD0E42918BFF329C5
:1007300007D0DE2918BFDF2903D0E82918BFDB293D
:1007400002D1204601F02CF805B030BD2DE9F84368
:10075000804602F019FBE725DFF840793C68461E29
:10076000B6414FF00009F60F02E0A14654F8084CDC
:100770009CB1607E0106F8D5207D012802BF94F867
:100780003D1098F804008142EFD14A462146384690
:1007900002F0C6F9B87A411EB9720EB102F0F0FA51
:1007A0003CB12046FFF744FEF021204600F0F8FF60
:1007B000002529464046BDE8F44300F0F1BF0000A3
:1007C00038B5054684B06878F32818BFDF2822D0F2
:1007D000E82818BFDB281ED0284600F029F80400BE
:1007E00018D1287CB0B105F11101092000F087F97A
:1007F00080B100F015F8A97A009101A92B89FFF7C3
:10080000FEFC0446F32C18BFDF2C03D0E82C18BFE5
:10081000DB2C03D16C70284600F076F805B030BDB3
:1008200002218DF80C104FF6FF72ADF804207047CE
:1008300038B504460025A07A0B381328207B28BF42
:10084000E8251028A8BFE82501DA0F2805D0DFF831
:100850006C140A7A110758BFE825617B884202D2DE
:100860000F2918BFE825DFF86C03418D4FF6FF72A2
:10087000914208BFEC25242001F092FFDFF89C1C78
:10088000086120B12422211D02F026F800E01A257B
:10089000284632BDA64D002070B50446CD4D207AC5
:1008A000DFF8706B6873607A85F82C00E07AE87086
:1008B000A07A307002F0D0FC307838B1211D502081
:1008C00002F040FEA11DE12002F03CFEDFF8C81757
:1008D000012081F8200004F10D01687BDFF83C5C09
:1008E0000F2814BF0120002028750B2205F11500E8
:1008F00001F0F2FF04F1180105F12000BDE870409D
:100900000B2201F0E9BF000010B50446607820B961
:10091000DFF8081C0869FFF7BFFF2C212170204673
:10092000BDE8104000F08CBF10B5DFF8F01B0446A6
:10093000086918B100220A6101F09CFF08202070AC
:100940002046BDE8104002F043BB0000DFF8481726
:1009500091F82000002800D1704780B5DFF85818C2
:10096000087D50B99B48C27890F82C10407BFFF767
:10097000F1FC10B1BDE80240F1E201BD30B5054621
:1009800089B0A87B0124410721D5E98E05F11C001F
:10099000FFF776FDD8B9DFF8A41C4879012808BF15
:1009A000002414D00B2205F10F0106A801F094FFDA
:1009B00000F08EFDACBF0321022106A83022019079
:1009C000009205F11C02EB8E012001F0A1F910202C
:1009D0008DF8080005F11C010DF10A0002F0B5F9CF
:1009E000E88EADF814008DF8164002A802F0F0FA77
:1009F00009B030BDDFF81C1A0878002818BF01F0D4
:100A00006EBB7047AD4800F154010162DFF8301C45
:100A1000416200F1440181620FF220010164DFF8BC
:100A2000241C0166DFF8581C8167DFF8581CC16779
:100A3000018941F002010181704700000304710443
:100A4000020460041104700402040204010402049C
:100A50001004610400041404630473047204620447
:100A600043040004130406040004000404041204F4
:100A700000040004000400045104640000040004A5
:100A8000000444040004000400040004650400049D
:100A9000350481046400050400048304000400009C
:100AA00002461146032000F010BF0146082000F066
:100AB000EEBE1CB5DFF8E4450FF2592060640FF27A
:100AC0003D20A06406E0204602F001F80090684650
:100AD00000F0BFFF21680029F5D1606838B1201D02
:100AE00001F0F5FF0090684600F0B3FFF5E72060E5
:100AF000A072E07220730FF2C950E06213BD38B5E6
:100B000004460FF2C050055D284601F02DFF20B1CC
:100B1000411941600021017232BD022001F024FF21
:100B200058B10FF2C451095D01701A21417001469C
:100B3000DFF86805007C01F038FF002032BD831D1E
:100B4000C907DBB20DD50A2193FBF1F10A2202FBA2
:100B50001131C9B229B10A335B1A0529A8BF0A337A
:100B60000B331328ACBF14200620C318DBB20933A3
:100B70000A2093FBF0F0C0B2704780B54F48017A6D
:100B8000880704D502F01CFB10B1012002BD002033
:100B900002BD4A48017A880781B00CD5B54A907ADF
:100BA00038B9DFF8F414C86F28B1407E10F0800027
:100BB00002D0012000E0002001B07047AD49DFF80D
:100BC0007C3A0A7B99788A4238BF01F0CDBE00207A
:100BD00070470000804D002080B500F03AFF0020F3
:100BE00002BD31B582B0017BA24C21B1012926D0D2
:100BF000032926D037E0DFF8445C687B0F281EBF4E
:100C00002E498A7A032A02D00298E16B884702991A
:100C100095F83A008873142002990870201D0299F3
:100C200001F03AFF02F0B0F8217BFFF70CFD2173D1
:100C300008B102F0A5F8202000F0ACFD37BD15206A
:100C4000EAE70146087A70B14868401C486002999A
:100C500010F8012D4A73029AD07D0028507B06D0EF
:100C600008B10A2813DB02A800F0F3FE37BD48B133
:100C70000A2807DA0FF25845137A291811F8011CCF
:100C80008B4204D0082804BF117A0829EBD1104602
:100C9000017A4A1E02720299487B0A300870029853
:100CA000417B491C4173B9E7DFF8F003C06C82B0A7
:100CB00008B102B0004702B0704700004443002072
:100CC00038B504460120207504F13C004188638F4B
:100CD000E18204F130020179E17641792177C1792D
:100CE00084F820100178204600F060FF050004BF62
:100CF000204600F034F9284632BD0000DFF8440CED
:100D0000817A032901D1202070470120704700001B
:100D100095172000417E41F001014176704710B5E2
:100D2000027D017E012A06D10B0704D44178BDE87B
:100D3000104000F035BD4C06DFF8603304D5407834
:100D4000196CBDE810400847012A03D1090748BFC4
:100D500030210BD441781B2908BF222106D000295D
:100D60000CBF0FF278310FF28031895C01700146BF
:100D7000BDE81040187C01F018BE70B5C64C0646A0
:100D8000E06F002872D03100DFF8AC5C04D01B2E7D
:100D900005D1017D052953D00022427052E0E92E91
:100DA0002ED1807E30B902F014FA18B1E06F817D47
:100DB00048072ED5EE2002F015FDE16F887EE8B1E0
:100DC0008A7D530705D4401E8876BDE8704002F046
:100DD000E2BD087E00F07F000876E06F017D032908
:100DE00003D1427E42F004024276ED2002F0FAFC8A
:100DF000DFF8501BE06FCA6F904726E04E7021E08D
:100E0000E12E15D102F0E5F9D0B1E06F817D480700
:100E100016D4E16FA87C8876E16F4A6828789070D4
:100E20002878401C28700120BDE8704002F011BDF8
:100E30001C2E05D10F490A6D90470020E06770BD58
:100E4000E06F4670E06FFFF76AFFE06F817D080694
:100E500005D5287E02F051FAE87D02F016FA00204E
:100E6000E0671020BDE8704000F094BC70BD000049
:100E70009D500020044F00202DE9FC4101F084FF2B
:100E8000854E441EA441F06FE40F00284FF0000887
:100E90005FD1824FB86C80473D6840F0100002E09F
:100EA000A84655F8085C002D53D0697E0140814268
:100EB000F6D142462946384601F032FEF567697E92
:100EC00008062CD4F87A411EF9720CB101F058FFD3
:100ED000F46FE18A207AFFF732FE3881A07D0106A7
:100EE00006D5E07E02F009FAF06F007F02F0CDF93E
:100EF000F26FD08AC10520D5398900291CBF92F82C
:100F00002000002811D090FBF1F082F82100F06F52
:100F100010F8081F1329ACBF0221002103E0B87AA2
:100F2000411EB972D1E7817605E0012082F82100E7
:100F3000F16F81F82200032005E0107E400800F0E8
:100F4000010080F00100BDE8F64102F082BCBDE87E
:100F5000F381002CFBD0BDE8F34101F011BF38B59F
:100F6000044600F06FFD217EDFF8D0060A0704D4A6
:100F7000217D012908BF027800D04278474D2146E3
:100F8000284601F0E9FDD8B1696C20468847A07D6C
:100F900041070ED401F0F8FEE97AFFF754FBE9723D
:100FA00008B101F0EDFEE08AC1050FD4BDE8314083
:100FB00062E7DFF890198A6F2046BDE8324010479B
:100FC000F12060702046BDE83240A8E631BD000047
:100FD000A850002050E738B50446DFF868090089BA
:100FE0000021820704F1380303D49A79550748BFDA
:100FF000E82110F0600F03D19879820748BFE821FB
:10100000DFF8A40B8279207A82421A7938BFE8216E
:10101000002A02BF18780028F52107D0080003D164
:101020002046FFF74DFE0146080000D038E031BDF4
:101030000D21017001F0CCBF38B5044600202070AE
:101040006070DFF8F815E08F0978144D420704D47A
:10105000EA7A8A4204D3F12122E0AA7A8A42FAD2B9
:10106000C10510D594F84210052912DB10F0050FC8
:101070000FD105F1240001F03AFB94F8421005F17C
:10108000240001F01BFB287C2146BDE8344001F020
:101090008CBCE821E0E70000C4420020044F00209F
:1010A0002046BDE834407BE310B504465C3080B296
:1010B00001F05AFC18B100F15C010472416010BDEE
:1010C000DAE6000000464A4C4449494339513A00A7
:1010D000020402010101010902000000303016186B
:1010E0001920231A1C1E3000303017181921301B0C
:1010F0001D1F3000DFF8080C0FF26511016000229F
:101100000FF2813141600FF2DD1181600FF2152184
:10111000C1600FF2113101610FF2C52141610FF27F
:101120009D2181610FF2B931C1610FF20941016264
:101130000FF2594141620FF2914181620FF2192180
:10114000C1620FF2E90101630FF2CD0141630FF2B9
:10115000C92181630FF25941C163DFF8A81B016403
:101160000FF27D4141640FF2ED418164DFF8980B8D
:1011700000F15C010A70CA7002220FF2196140F896
:101180003C1F01610271012101757047F8B502220F
:101190008DF800208DF8010008B14FF6FF71ADF811
:1011A00002100B22DFF8641B01A801F095FB6846D2
:1011B00001F00EFF05B000BD8850002080B50A2266
:1011C0008DF801008DF800208DF80210684601F0BE
:1011D000FFFE01BD3EB504460120E08204F132016C
:1011E00002202075684601F0B0FD6068A38F94F876
:1011F0003E10401E606001706A46207A401C2072DA
:101200008321204600F0D2FC050004BF2046FFF7F2
:10121000A6FE28463EBD0000DFF8202692F83510D5
:1012200030204143DFF8700C01F048BA30B5DFF8E8
:101230000C46607B0F2893B006D02E218DF800104D
:10124000684600F0FDFA09E000F0DEF8608E142137
:10125000B0FBF1F105F1340001F030FA13B030BD0C
:1012600038B504466078010032D104F13205297A9C
:1012700002291CBF0329E82094F82F100B391329E9
:1012800013D2010024D104F12F01E12002F05AF918
:1012900004F13C01502002F055F9297ADFF89C0551
:1012A000022904D12A88028408E0E82012E04FF6DF
:1012B000FE7101841630294601F05FFD0B2204F116
:1012C0002401DFF8480A01F007FB2046FFF782FF00
:1012D000010006D06070172020702046BDE8324023
:1012E000AEE231BD18B5DFF8204A94F85F0085B052
:1012F000A8B9012184F85F10012002F06CFC02A85B
:1013000000F0F1FBDFF8342504F1540001210190D5
:1013100000910321D38C02AA052000F0F9FC06B04D
:1013200010BD000010B500F0A9F82178202904BFF5
:10133000EB20607000F0ECF844BF01F0FB0180F896
:101340005F1000F0E1F800D5EAE02A202070204686
:10135000BDE8104074E200007CB500F08FF800F0AA
:1013600053F805F1440001F0C2F900F06DF9ADF851
:10137000001060688678300008D16946532002F07A
:10138000E1F804F11C014A2002F0DCF80B2204F120
:101390000F0105F1540001F09FFABDF8001030462E
:1013A000FFF7F4FE95F85F00810703D56078002110
:1013B000FFF704FF002085F85F0073BD10B50446F9
:1013C000EB206070DFF8800B90F85F20900703D56A
:1013D0000021EB20FFF7F2FE4FEA0400BDE81040C9
:1013E00038B500F04BF800F00FF805F1440001F0BB
:1013F0007EF905F15C0000210170C1704FF6FF71AC
:101400006078BDE83440C1E6DFF83C5B05F13400AC
:1014100001F06DB9F44F002010B50446FFF7CEFF80
:10142000CCE0000010B500F029F8207A002814BFA5
:101430000020EB20607000F06BF844BF01F0FB016E
:1014400080F85F1000F060F80BD501F0FD0180F826
:101450005F1000F095F8ACBF01210021FFF7AEFE50
:1014600008E0C80706D52A202070EB2060702046CF
:1014700000F0E6F92046BDE81040D9E50446012019
:1014800002F0BABB1CB50446DFF8BC0A90F85F1046
:1014900041F0020180F85F10012002F09CFB6178AE
:1014A00079B900F015F8ACBF0321022104F1100056
:1014B000012201900092221DE389052000F028FC02
:1014C0006070607818B1BDE81C40002176E613BD5D
:1014D000DFF86803418D4FF6FE72914270470000BD
:1014E00010B5FFF7CBFF2178202904BFEB206070F7
:1014F00000F00EF844BF01F0FB0180F85F1000F02F
:1015000003F800D50CE010BD90F85F108A07704713
:10151000DFF8340A90F85F104A07704788500020BF
:1015200001F0FD0180F85F1000216078BDE81040F7
:1015300044E6000038B5FFF7A1FFFFF765FF207A0A
:10154000002814BF0020EB20607095F85F00410771
:1015500044BF00F0FB0085F85F0095F85F0081074D
:101560000AD500F0FD0085F85F0000F009F8ACBF77
:1015700001210021FFF722FE2046BDE8324057E559
:10158000A07B00F0100001286078704710B5FFF7CD
:1015900075FFEB216170FFF7BBFF44BF01F0FB015A
:1015A00080F85F10FFF7B0FF00D5B9E710BD00006D
:1015B00010B500F010F82046FFF7E8FF2046BDE820
:1015C000104000F01BBD000010B500F004F82046EC
:1015D000BDE81040DAE70446DFF8EC0B01F087B80D
:1015E00018B5044685B004F11C01DFF8E00B01F0EA
:1015F00099FB08B3EF2009218DF801008DF8001048
:1016000000F022F8ADF80210606801798DF804103E
:10161000207A082804D16168C8798DF8050002E0B5
:1016200000218DF8051004F10F010DF1060000F006
:1016300013FC684601F0CCFC06B010BD54F9210043
:10164000B45000200101200060680178407801EB6F
:101650000021704700F043BDBA48DFF8A41681614D
:101660003831C1610FF2200141630FF280018163C3
:10167000DFF8601BC165018941F0010101817047FC
:10168000AD052000010620000101710101010101E9
:10169000110101013101010101018001100161010C
:1016A0003B001400630173017201620143010001F8
:1016B000130106013D013500040112010001000182
:1016C0000001000104010401330133013C01440124
:1016D0003201360000010001650100013500810181
:1016E0000001050182018301000100000302710273
:1016F0003001600211027002010202020202800245
:10170000100261023A004100630273027202620237
:101710004302000213023800000200020402120217
:101720000002000200020002040204023700370037
:101730003C0244020002390000020002650200027D
:1017400035028102000205028202830200020000CB
:10175000024611460220B8E00146062097E01CB57B
:10176000784C206810B1204600F073F90021A17276
:10177000DFF8381B086858B102E0684600F069F9E4
:10178000DFF82C0B007C01F03DF900280090F4D12B
:1017900013BD00000146DFF8180B007C01F0FEB914
:1017A00000B585B003780FF27C02D25C8DF8002082
:1017B0000B2A03D1417000F071FB31E082B30C2A97
:1017C00029D11A2902D10020019024E0019090F83B
:1017D0003D208DF80220C2680292028AADF80C20EA
:1017E000827DD30648BF002204D4144A92F83430D4
:1017F000827E9A1A8DF80E20427F8DF80F20827F0C
:101800008DF81020C27F8DF81120C08AC20544BF18
:1018100011228DF800208DF80110684601F0D8FBE8
:1018200005B000BD0C0E020B040B0A0708000F00E8
:101830009748817A481E8041C00F7047804D002034
:1018400038B5934A937A02F1300102F1300551F82C
:101850002330017801F07F01017003EB41014C78E6
:10186000214655F8211001B19472047813F8143010
:10187000190902EB8102D16811B9BDE83240F0E2EA
:1018800003F00F0351F82310BDE8344008477CB53E
:1018900005460FF28400405D0E4601F065F8040035
:1018A0000CD0257000210FF27C0061703146425D42
:1018B000201D01F011F800F03BF873BD8DF80050C9
:1018C0001A216846FFF76CFF73BDF8B507460FF2A3
:1018D0004800C65D0D46304601F046F8040012D0BF
:1018E0002770002060702946A019606000202072D7
:1018F0000FF23000C25D04F1240000F0EDFF00F0B3
:1019000017F80020F2BD8DF800701A216846FFF725
:1019100047FF1A20F2BD000000055957515C1C20FA
:101920002807020000011C181A18181C24030000C4
:10193000DFF87C09007C214601F037B8DFF8701928
:101940000874704744430020F8B50E46B006504D69
:10195000DFF85C7919D41DE001F016FA397B401EDE
:1019600080414A1EC00F3A7308B101F009FA20788D
:101970008DF800006C602046FFF762FF9DF80000C4
:1019800015281CBF281D00F064F8381D01F09FF8D1
:101990000400E1D1300406D40AE06860FFF750FF8C
:1019A000281D00F056F8387C01F02CF80028F4D1FE
:1019B000F00602D52D2000F041F8F00702D52420D2
:1019C00000F03CF8B00702D5252000F037F870078A
:1019D00002D5262000F032F8300702D5282000F08A
:1019E0002DF8700607D500208DF801002C218DF808
:1019F000001000F025F8300607D500208DF8010012
:101A00002F218DF8001000F01BF8286888B101F034
:101A1000BBF9401E2C6880410021C00F296008B12D
:101A200001F0AEF96C602046FFF70AFF281D00F0B8
:101A300010F80020F2BD0000A24D00208DF800003B
:101A40006846FDE612494A68824204BF00204860A9
:101A5000704738B5040008BF02F06CF901F094F942
:101A6000451EAD412168ED0F59B1094A5368A1F1F6
:101A700008008B4204BF002151600021216000F06A
:101A8000F9FE1DB1BDE8314001F07AB931BD000069
:101A900044430020DFF8600B0FF2C53141600FF2C4
:101AA000D13181600FF2CD31C160DFF8501B01618F
:101AB0000FF2E9314161DFF8481B8161DFF8701BEB
:101AC000C1610FF20D7181630FF29141C1630FF299
:101AD000ED4101640FF2815141640FF221518164A3
:101AE000002101707047DFF8901B0A8C4FF6FE73DF
:101AF0009A4204BF163101F028B902220272098C01
:101B00000180704742784B78C2F38102C3F38103AE
:101B10009A4211D1022A09D142794B799A4202BFE5
:101B200080798979884207D101207047032A03D13F
:101B3000491D401D01F013B90020704738B5547895
:101B4000057A0023C4F38104AC4218D1022C10D1D1
:101B500054799579008804EB0524A4B2A0420ED1F3
:101B6000D078127900EB022080B2814207D10123A4
:101B700005E0032C03D1511D01F0F1F8034618468E
:101B800032BD017ADFF8F02A022907D1128C0088D1
:101B9000824201D10120704700207047014602F1C6
:101BA000160001F0BFB8000054F921002DE9F84FEC
:101BB00090469946DFF8C02A98F8084002F11406CA
:101BC0000B064CBF4FF6FF77778A054601F07F0181
:101BD0008DF800104FF0000AA87D81064CBF082048
:101BE00000202876A87D41074CBF80201020687611
:101BF00002F13400A97DCB064CBF00210178A97603
:101C0000E98ACB0748BF4FF0200A090769682B7D96
:101C100048BF4AF0100A491E022B07DB0B2B1CBFE2
:101C20005B1E01F801394AF0030A01E043EA0A0A9F
:101C3000407D012804D12B7A672BA8BF4AF4805A33
:101C40009DF8000002284AEA803A07D1F08A000A8B
:101C50000870F28A01F8012C891E0AE0032808D1D5
:101C6000A1F1070B02F13C01584601F086F8ABF1F7
:101C700001019DF8000050B124B14F4508BF4AF062
:101C8000400A04D03812087001F8017C891E022C29
:101C90004AEA842A09D1B8F80000000A01F80109CB
:101CA000B8F8002001F8012907E0032C05D1CF1F67
:101CB0004146384601F061F8791E2CB14FEA1920EF
:101CC000087001F8019C891E287D4A1E18B93078D9
:101CD000431C337002E0B07B431CB37308704FEABF
:101CE0000A40000E107002F801AD297A68686A6037
:101CF0004118891A297200206870BDE8F28F00002F
:101D0000A84F0020492420004C4E0020A04E002067
:101D10002DE9F047099D894607469246984629468F
:101D2000FEF7EDFE1A2604001AD00898E082277507
:101D30000B22294604F1240000F0CEFD4346524612
:101D400049462046FFF732FF064648B9FF1F012FDC
:101D500003D8607E40F0200060762046FFF7FFF851
:101D60003046BDE8F0873EB5044604F13C0501214C
:101D7000687800B105210420E182207504F130016A
:101D8000684600F0E2FF6068638F401E60606A464C
:101D9000297801700321207A401C20722046FFF729
:101DA00005FF050004BF2046FFF7D9F828463EBDD1
:101DB00070B504460D460520207005F13A06F0780E
:101DC000A0706068296B416105F11C0100F0BDFF46
:101DD0006068E98E41813178417400216068017644
:101DE000C17305F10F016068193000F035F86168C2
:101DF000A87B88736868626801789181437841EABA
:101E0000032191818178C01CCB0918BF0123137471
:101E100011F0070201F0070118BF012201EB410197
:101E20005118C9B2084410F8011B2172E060217AF0
:101E30004A00490802F00E0201F0380189180844EE
:101E40006061297A6A685318834227BF081A1018FC
:101E500000202072207470BD0B2200F03DBD0000F8
:101E6000704701780B29BCBF1821FFF799BC704758
:101E7000192195E438B5DFF8B0580446286828B130
:101E80001921FFF78DFC2846FFF7E3FD2046FFF7F9
:101E9000D9FD2C6031BD0000904E002030B50446C5
:101EA00089B02078DFF88458032808D0052812D09C
:101EB000182804D01E2818BF1F280CD01CE00020B2
:101EC0008DF8180004F12F0103A800F056FF03213C
:101ED0008DF814100AE001218DF8181003A804F100
:101EE0002F0100F04AFF03208DF8140000F02EF8B7
:101EF000E88CADF8160015E002218DF8181003A843
:101F000004F11C0100F039FF03208DF8140000F0EB
:101F10001DF804F10F01E88CADF816000DF1190061
:101F2000FFF79AFF0B208DF800000DF11900617882
:101F30008DF8011004F10F01FFF78EFF684601F0E4
:101F400047F809B030BD00004C4E00200221688DDA
:101F5000ADF802008DF80A107047000038B504464D
:101F60006578280014D1DFF81017608FCA8C904272
:101F700018BFE82504F13000FFF703FE90B10021FF
:101F800084F83D10280003D12046FFF7ECFE0546FB
:101F9000280006D06570192020702046BDE8324028
:101FA0004EE431BD94F83D000028EBD0DFF88017F7
:101FB00091F820000028E5D1E825EBE718B585B0B9
:101FC00004218DF8041000F1300142788DF80520CD
:101FD000428FADF810200DF1060000F0B6FE0DF1B5
:101FE0000600FFF7CEFD20B100F02DF8DFF83C072A
:101FF000048401A800F0ECFF06B010BD18B587B04E
:10200000044603208DF8040004F11C010DF10600C4
:1020100000F0B3FE616808788DF80E0004F10F013E
:102020000DF10F00FFF718FF04F11C00FFF7A9FDE9
:1020300020B100F008F8DFF8F406048401A800F0ED
:10204000C7FF08B010BD4FF6FF74ADF800406946F9
:10205000532001F077BA000030B5054691B06868AA
:10206000DFF814464178480609D5E08CE98E8842AD
:1020700005D1DFF884150878D0B100F030F808A950
:10208000039102A82946FFF793FE2B208DF8080044
:1020900002A8FFF7D5FBA07810B19DF8180028B171
:1020A00005218DF8081002A800F092FF11B030BD94
:1020B00094F830000028E2D005F11C00FFF761FD24
:1020C0000028DCD105F10F0001210190009104F1FD
:1020D0001602E38C03210620FFF71AFEE6E700B59F
:1020E00085B009208DF80000EE218DF801106846BA
:1020F00000F06EFF05B000BD2DE9F041054600F08F
:1021000043FE441EA441E40F0DB101F0DDF9DFF8F8
:10211000685501F04AFB05F1390600277078DFF8B1
:10212000088601F0EAF83078DFF8CC6401F0ADF809
:10213000307801F091F8E88C01F099F8688D01F0A1
:1021400098F805F13C0001F09BF808F15C0050F8AC
:10215000270000B180477F1C072FF6DB00F0E5F970
:10216000FFF7FDFA00207070FEF7A3FCFFF792FC6A
:1021700005F12901522001F0E5F90CB100F000FE53
:102180000020BDE8F081DFF870040FF26901016200
:10219000021D0FF23D3141620FF26D3181620FF28B
:1021A0001511C1620FF2052101630FF2BD114163E8
:1021B000DFF87415CA6000F13802203048610A6106
:1021C0000020088101F0E2BA804E0020964D0020E8
:1021D00070470000F5102000072202700A7A827012
:1021E0008A7AC2704A68426000220272C969C1607C
:1021F0007047000038B50446DFF838550020687095
:10220000207A0628A4BFE8216970607A0E2804DDD0
:10221000217A032904D0E8206870207A032806D1A7
:10222000DFF80415087AC1075CBFE8216970214610
:102230002846FFF7D1FF6068800A286205F1240074
:10224000617A0170E17A4170217B8170617BC1709C
:10225000A17B01710A214171DFF81C1491F83A2029
:1022600082710B22DFF8D004A86104F10F01042071
:10227000287705F12B0000F02FFB6978002904BFB7
:10228000607800280BD1A87808B1EA21697001F0C4
:1022900076F826202070042001F087FC01E0292038
:1022A00020702046BDE83240FFF7CABAA054002093
:1022B000044F002078B5DFF87C440546A07885B04F
:1022C00070B994F829100A290AD001F081F8E16860
:1022D00094F82920114401F80B0C207A401C20723C
:1022E000216A94F8290049082162401CC90784F832
:1022F000290002D4C1B21E29F2DBC0B21E282CD0A4
:1023000004F12901E12001F01DF902208DF81000EF
:102310004FF6FF73A078ADF80830002818BF0228E8
:1023200003D1284600F020F81CE0012804F12B021C
:1023300007BF0820802107208321019200260096F4
:1023400002AAFFF7E5FCDB2818BFE52804D0F32834
:102350001CBFDF28E82805D1607029202870284696
:10236000FFF76EFA06B070BD38B5DFF8C843606895
:1023700004F1240101254A7905FA02F290436060D4
:102380003022A078032804D1DFF8A03393F8355029
:1023900002E009788D406D1C554308B901F016F82C
:1023A000294604F11000BDE8344087E1F0B5DFF8BC
:1023B00084530446A87802281CBF012805288FB042
:1023C0003CD1002006A96870019168462146FFF7BC
:1023D000EFFC2E7A95F8250086421BD2EF680BE0C1
:1023E0007889BDF82210884204D106A9384600F049
:1023F00099FC78B9761E2437F0B20028F0D12E7AF5
:10240000EB682422564306A9981900F065FA297A48
:10241000491C2972DFF81423907828B19DF8101018
:1024200011B995F8250010B9684600F0D1FD95F86E
:10243000250038B1297A814204D101E0E820687092
:1024400000F040F80FB0F0BD7CB5044604F1240064
:10245000DFF8E0520178032904BF827A032A2CD1E5
:1024600004F11C014A2001F06DF86068017842789F
:1024700001EB0221ADF80010861C6946502001F0E6
:1024800061F83078717800EB0120ADF80000694602
:102490004B2001F057F8B61C3146E12001F052F80C
:1024A000701C0178407801EB0021ADF8001053203A
:1024B000694601F047F8002000E0E820687000F06D
:1024C00001F873BD292020702046FFF7B9B900003C
:1024D00010B5DFF8604204F1100000F008F900F0D8
:1024E0006BFF042001F088FBA178032904BF60780A
:1024F000002804D004F12A01E12001F023F820464D
:10250000BDE8104000F064BDF8B501466846FFF72D
:1025100063FEFC218DF80110684600F059FD05B0FE
:1025200000BD01460720FFF7B2B9844800210160D1
:1025300041604FF47F018160C160002101617047FB
:1025400038B57E4C00202061206868B14068A168E1
:10255000884209DA01F02BFC21684D68A842B8BF17
:1025600028464860206820612069616831B118B14F
:102570004A684068824202DA216100E040B1206985
:10258000A1684068884203DABDE8324001F037BCF8
:10259000BDE8314001F059BCF8B500F0F5FB674DDE
:1025A000441EA4412869E40F10B3A9684068814221
:1025B00003DA01F0BFFB2869D0B101F0F8FB29690B
:1025C0004968884214D3002948BF01F0B3FB2F6942
:1025D000384600F08CF83E7BBF680CB100F0D0FBB1
:1025E0003046B84700F0D0FB441EA441E40FE2E7B8
:1025F00004B195E0F1BD0000F44F0020D70F20009A
:10260000D50F200070B505460C464C4E0DE06068B5
:10261000316928188C4202D1002848BF0020606030
:10262000002848BF01F086FB2468002CEFD170BD64
:102630003110200070B5414E00F0A6FB746831687F
:10264000451EB068AD414042FFF7DCFFB168ED0FB9
:1026500005E060688842A4BF401A60602468002CCE
:10266000F7D1F06881421CBFB06001F087FBFFF733
:1026700067FF05B11EE070BD804D002070B50446B7
:102680000D4600F081FB461EB6412868F60F29462C
:1026900030B1626843689A42A4BF01460068F7DA25
:1026A0000C6020602868A04208BFFFF749FF06B110
:1026B00000E070BDBDE8704000F062BB38B5044674
:1026C0000D4601F074FB451965602046BDE83440B5
:1026D0001A49D3E70A6801E011461A462AB113687D
:1026E0008242F9D10B60012070470020704770B51D
:1026F000044600F049FB114E451E31462046AD41CF
:10270000FFF7E8FFED0F18B9311D2046FFF7E2FF94
:102710003069844208BFFFF713FF05B1CAE770BDF7
:10272000BDE8F14000F02CBB44430020804D002068
:10273000C44200203C51002095172000C4430020D3
:1027400010B56148614B41F2FC7200218152186062
:102750004FF42774048000F5277048F2040141F219
:102760005C520180828010BD38B5012000F018F85D
:10277000050008BF01F0DEFA00F006FB5349441ED5
:10278000A441281F0860E40F284600F073F8504960
:10279000012008701CB1BDE8314000F0F1BA31BD34
:1027A0002DE9F84300240026051D15F003001CBF89
:1027B000291D0D1A00F0E8FA444FD7F800C0431E57
:1027C000434800789B41DB0F10B1A9B2112907D211
:1027D0006246D2F800E0CEF3C03119B1002627E0FE
:1027E0003C4AF6E7A9B2EEB1D4F80080C6444FEAFD
:1027F000D839CEF30E0E4EEAC93EC4F800E0CEF34F
:102800000E0E8E4514DB44B32268C2F30E06761B0F
:102810001FFA86FEBEF1080F13D3665245F4004539
:10282000258011E0CEF30E048C4221DA01261446F5
:102830001168C1F30E010A4411880029C9D100248E
:102840000BE042F40042226030B1A44504D120687C
:10285000C0F30E0021183960241D0BB100F090FA6E
:1028600014F0030018BF01F065FA2046BDE8F283BA
:102870001446C8E710B514498842044603D301F54D
:10288000C051884201D301F055FA54F8040CC0F34A
:10289000C03008B901F04EFA00F076FA54F8041C82
:1028A0000A4A21F40041401E44F8041C8041136888
:1028B000C00F211F994238BF116018B1BDE8104008
:1028C00000F05EBA10BD00002C55002030770020CB
:1028D00010550020CC57002003E011F8013B00F810
:1028E000013B13465A1E002BF7D1704710B5134613
:1028F0005A1E3BB110F8013B11F8014BA342F6D030
:10290000002010BD012010BD10B5044610460A4637
:102910000146204601F0AEFA204610BD0146087877
:10292000497800EB012080B27047024602291078F6
:1029300003D1517800EB01207047032906D151786B
:10294000927800EB012000EB02407047042908D187
:102950005178937800EB0120D17800EB034000EB35
:102960000160704701F00EBB10B5040001D10020DA
:1029700010BD04F1080080B2FFF712FF28B100215A
:102980000160FF2284808271083010BD80B508B9D3
:10299000052002BD10F8021CFF2901D0042002BD51
:1029A0000838FFF767FF002002BD0022FFE738B5B7
:1029B0000446A1B1DFF858331D78A84204D3084675
:1029C000FFF7E4FF032032BDA1F1080318680028D7
:1029D00004BF9879FF2804D00846FFF7D7FF0520E9
:1029E00032BD012A9C71DFF82C0302D100F087F878
:1029F00001E000F051F84FF40041204600F0CEF81D
:102A0000002032BD2DE9F041804600F0BDF90026DE
:102A10000024DFF80053471EBF412868FF0F58B15C
:102A200010F8021C414502D01CB9064601E0A4B9C9
:102A3000044650F8080CF2E74FF40041404600F01D
:102A4000C4F824B132462146284600F069F80FB197
:102A500000F096F92046BDE8F0814FF40041404671
:102A600000F09CF8EEE770B505460E4600F08CF9D4
:102A7000A8490C68401E8041C00F44B114F8021CE4
:102A8000A94206BF2378B34254F8084CF5D108B1E7
:102A900000F076F9204670BD38B500F014F8421EFB
:102AA0009241002045F8080CD20F216811B9256029
:102AB00006E0014651F8080C0028FAD141F8085CFC
:102AC00002B129E031BD04460D4600F05DB938B5CC
:102AD000044600F059F90025411E89412068C90FBC
:102AE00040B10546A5F10800002302682260FF24DA
:102AF0000360847109B100F043F9284632BD38B54E
:102B0000FFF7E1FF401E216845F8081C8041C00F17
:102B1000256000D000E031BDBDE8314000F030B9A3
:102B200070B504460D46164600F02EF9401EA5F17C
:102B30000801804123680A68C00F9D420CBF2260D3
:102B400046F8082C0022FF230A608B7118B1BDE8FB
:102B5000704000F015B970BDF8B506460D46174631
:102B600000F012F90024431E9B413168DB0F09B9C4
:102B700035600DE07A1E03E0D1B251B10146521E1C
:102B800051F8080C0028F7D1D2B212B141F8085C14
:102B900001240BB100F0F4F82046F2BD38B500F086
:102BA0002CF810D200F0F0F85B49096831F81420D5
:102BB000401E8041154321F81450C00F08B100F0A9
:102BC000DFF8002032BD032032BD38B500F015F823
:102BD00011D200F0D9F85049096831F81420401E8C
:102BE00022EA0505804121F81450C00F18BF00F0FB
:102BF000C7F8002032BD032032BD0D4644490A7893
:102C000090420446704780B5FF2803D100F0B8F821
:102C1000002002BD072002BD80B5FF2803D100F0CF
:102C2000B3F8002002BD072002BD80B5FFF788FD84
:102C300038490020086001F0A7F901F09BFA01F083
:102C4000A3FAFFF791FD002002BD80B500F001F866
:102C5000FCE72DE9F04101F009FB2D482E4C0178ED
:102C600000262268F3B232F8130018B9761CF2B2CB
:102C70008A42F6D3F0B2884229D200F085F8216862
:102C8000F5B231F81580401E8041002221F8152050
:102C9000C00F08B100F074F8204F214A3E70414641
:102CA00052F82530F0B298470646FF20387000F001
:102CB0006BF8216831F81520401E8041164321F839
:102CC0001560C00F18B1BDE8F04100F059B8BDE87B
:102CD000F08101700A0A0B0C090E42708370C170FA
:102CE000001D704701700A0A090C42708170C01CF7
:102CF000704710B540B1002300E05B1CDCB2944289
:102D000004D2045D8C42F8D0002010BD012010BD1B
:102D1000363D20009C540020A05400200544002093
:102D2000EC412000027A0B7A9A420CD15AB1022A65
:102D300005D100880988884205D101207047032AFF
:102D400008BF00F00CB8002070470A7A0272032A0C
:102D500004BF0822FFF7C0BD0B880380704710B581
:102D6000082210F8013B11F8014BA34203D1521E77
:102D7000F7D1012010BD002010BD0822FFF7ACBD27
:102D800080B501F079FA02E080B501F071FA00B186
:102D90000120C0B202BDF0B54F4C504A25689542A3
:102DA0000AD02568002605EB86073F6842F82670A2
:102DB000761C402EF7D3226042F82010F0BD10B5EB
:102DC0000FF22C12830852F823201368C00000F081
:102DD0001800FF248440A34381401943116010BDB3
:102DE00004283F4903D1086840F480300BE00528EF
:102DF00004D10A6842F400320A607047062804D100
:102E0000086840F48020086070470F2805D13548D5
:102E1000016841F00201016070470CD90FF2741390
:102E2000A0F110011038400953F82000012201F0F0
:102E30001F018A40026070470428294903D10868AD
:102E400020F480300BE0052804D10A6822F4003217
:102E50000A607047062804D1086820F480200860C2
:102E600070470F2805D11F48016821F00201016059
:102E700070470CD90FF23013A0F11001103840093F
:102E800053F82000012201F01F018A4002607047C0
:102E90000E28154904D1086840F0006008607047AA
:102EA0000F2804D10A6842F000720A6070470CD9FA
:102EB0000FF20813A0F110021038400953F8200057
:102EC000012102F01F02914001607047074801682C
:102ED00041F001010160704708ED00E00040002072
:102EE00024ED00E010E000E004ED00E098200D404B
:102EF0000000000018ED00E01CED00E020ED00E017
:102F000000E400E004E400E008E400E00CE400E099
:102F100010E400E014E400E018E400E01CE400E049
:102F200020E400E024E400E028E400E02CE400E0F9
:102F300030E400E034E400E038E400E03CE400E0A9
:102F400040E400E044E400E048E400E04CE400E059
:102F500050E400E054E400E058E400E05CE400E009
:102F600060E400E064E400E068E400E06CE400E0B9
:102F700070E400E074E400E078E400E07CE400E069
:102F800080E400E084E400E088E400E08CE400E019
:102F900090E400E000E100E004E100E008E100E08E
:102FA0000CE100E010E100E080E100E084E100E0FD
:102FB00088E100E08CE100E090E100E080E200E0E8
:102FC00084E200E088E200E08CE200E090E200E0D1
:102FD0002DE9F14382B0067892A18D5DADF80050E5
:102FE000002D4AD00D2E4FF6FF7911D1694653209E
:102FF00000F088FABDF800004FF6FE7188421FBF4E
:1030000048450299087A002800F0AB800C466DE034
:10301000052E4FF0240804D102990A7C243250195D
:103020000AE0072E0AD102998878002828460EBFA8
:103030001B300A7A08FB0200ADF80000BDF8000062
:10304000FFF792FC04001CD10C2E16D1029948689F
:10305000002812D0FFF798FE471E0298BF41001DBE
:10306000FEF7F7FCBDF80000FFF77EFCFF0F040041
:1030700004D1002F01D0FFF783FE96E00FB1FFF7D8
:103080007FFE02992A462046FFF726FC052E12D124
:103090006168242204F11800FFF71EFC04F11800F7
:1030A0006060227C61692430FFF716FC606800F1E3
:1030B000240161611AE0072E18D153480568ADB1AB
:1030C00000210160A07828B904F11001E1601B2201
:1030D000E06805E0217A04F1100008FB01F2E060ED
:1030E0002946FFF7F9FB2846FFF7C4FB474801686C
:1030F00019B12046884700284DD10D2E444834D1BF
:1031000002994A6813785278C3F3830103F00303EA
:10311000022B0ADA3F4B9D7CA94201BF12F0C00F7F
:10312000029A92F82430022B09D0032919D1029A6D
:103130000121117000780299FFF737FC35E094F80F
:103140003B0004F13A0100F046F80298C18C494571
:103150001CD141688879022818DB204601F09EFACC
:1031600018B302A8FEF775FC1FE00C2E1FD10298C1
:1031700041781A291CBF6068002807D0807DC107EC
:1031800004D5207C04F10F0100F025F822480078D6
:103190002146FFF70AFC0C2E18BF112E05D102990B
:1031A000486810B1081DFEF754FCBDE8F783112EE6
:1031B000ECD10021217021460078FFF7F6FBEEE705
:1031C00016480078002814BF012801F0ECB900204F
:1031D000704700207047124A1278A2B10B7832284B
:1031E000B8BF322002DB6F28A8BF6E20012A04D1AD
:1031F000323858433C2290FBF2F398B2B0F5807F0E
:10320000A8BFFF230B70704754540020BC5400200B
:10321000C8520020084D0020685400207842002049
:10322000225500200016100000181510020002247C
:10323000144000001014000075480B218170FF211C
:103240004170C1700170704780B500F0B5F8BDE8FD
:103250000140BDE001F03ABB6E490A68030018BFA7
:10326000012322F0020242EA43020A6070476A49DF
:1032700000E06A4900F0FF020A60000A48607047F7
:1032800001460822664801F0C3BC38B504466548CB
:103290000568297860B24AB28242A3BF69784BB20E
:1032A00098420C46FFF770FD2978594B401E80412B
:1032B000091B891CC9B2C00F6A5CDA7008B1FFF73C
:1032C0005FFD00F002F8204632BD38B5FFF75CFD27
:1032D0004F4AD3781478411E8941C90FA34209D0BF
:1032E000514D287830B9514C2078050602D4504809
:1032F0001370036001B116E031BD38B504460B38D8
:10330000122828BF00F016FDFFF73EFD4049474A4E
:103310008C70451EAD411078ED0F08B900F007F82C
:1033200005B100E031BDBDE83140FFF729BD10B562
:103330003E49087808B100F0FDFCFFF725FD344C4C
:10334000A1786278401E8041C00F914211D0617017
:1033500008B1FFF715FD00F0BBFC6078354900EBC4
:1033600080002C38086001F0B8FCBDE8104000F087
:1033700070BC18B1BDE81040FFF702BD10BD38B5F4
:103380002D490546087808B100F0D4FC2B4C207874
:1033900008B100F0CFFC28000CBF0120032D09D09C
:1033A000012D1CBF022D00F0C5FC1B49FF220A6045
:1033B00002204A60207031BD2049214A0020087057
:1033C0001549D08C00F0FF030B6056E701F0CFBB2E
:1033D00080B501F0D6FB1B4A1B49137803F00F039D
:1033E000C95C0818BDE80240493840B210F1570FD7
:1033F000B8BF6FF0560002DB0B28A8BF0A20573079
:10340000C0EB0020612190FBF1F0C0B270470000DA
:103410008C54002000860840C8850840D0850840AC
:10342000A885084040F921008652002098520020CB
:10343000408608403C860840024400208552002017
:10344000804D00200C55002044F92100CEE7F0B457
:103450000246106895681318506803EB5004C007C3
:103460001DD54D441BE013F8017B05F8017B491E77
:10347000F9D1A0B1B60813F8011B06F00306032E1C
:1034800008BF13F8016B01EB06214942801C294457
:1034900005D011F8016B05F8016B401EF9D1A3426C
:1034A0000ED013F8016B16F0030104BF13F8011BD3
:1034B000C91C30090F28DAD113F8010B0F30D6E7F9
:1034C000F0BC02F10C00704710B5664C67A12046B5
:1034D0006C2201F04FFF1434FFF7BCFEA073FFF71E
:1034E000B9FE207010BDA0F140021E2A38BF40383E
:1034F00004D3A0F1E0010F2902D23E30C0B27047E0
:103500002D20704770B50D46FFF7EDFF06462D2EB6
:1035100001D1F42070BDFFF737FC524BB0F101042C
:103520006DA000EB860110F826004A78A441191816
:103530002846FFF7D1F9E40F0CB1FFF721FC00207A
:1035400070BD00002DE9F041F12805460E46DFF878
:10355000148111D1317801290AD1022000F04CFBED
:103560002846FFF7C0FF2D28014612D1F42077E04E
:10357000022000F01AFBF3E7F02805D130783A4931
:103580000870FFF769FEEBE74528E9D1C8F8086045
:1035900065E000BF50A000EB8107B978002904BFA7
:1035A000F878002815D0F878814208BFFB2057D062
:1035B000582D05D130888F3846F22241884206D2F4
:1035C0003078B978884224BFFA78824201D2E82064
:1035D00046E0FFF7D9FB7A78441E387831464044FC
:1035E000A441FFF779F9E40F0CB1FFF7C9FB502DA7
:1035F00008F12A0010D0522D17D0532D11D0E02DF4
:1036000027D0E12D1CD0E22D1ED0E52D25D0E62DB2
:1036100004BF3278C27722E0B8F82600FFF727FE11
:103620001DE00088FFF725FE19E098F8290018B181
:10363000022000F0BAFA12E0022000F0DDFA0EE0FB
:10364000007CFFF75AFE0AE008F13C00FFF718FE85
:1036500005E0C07BFFF719FE01E03178817700209B
:10366000BDE8F081804D0020F44F002036000100BD
:103670000600000000000000000F00000000000035
:10368000000000000000000000000300FFFF000039
:103690000403FFFF0000FFFF0F00F4010005C40456
:1036A0000320000100000B000000000000000000EB
:1036B0000300010F000000000000000000000000F7
:1036C00000000000000000000000000000000000FA
:1036D000000000000000000000013636010100017A
:1036E00002010001030100010401060608040000B4
:1036F0000C0100340D01000F10040101140100FF42
:103700001608000020020000220100FF2301000132
:10371000240100FE25010008260200002801000106
:10372000290100012A0200002C01000F2E020000D6
:103730003001000131010008320200FF34010007AE
:103740003501024036010000370100013801000157
:10375000390100FF3A010B1D3C080000460100083A
:103760004701000F48010001490100FF4C0400001F
:103770005004000054040000580400005C040000E1
:1037800060040000640400006804000080B500F0DC
:10379000FDFFFFF751FD00F003FA01F06FFA00F0B2
:1037A0004FF8BDE8014000F0C7BA80B5FFF7ECFA6A
:1037B00018B9FFF7E5FA00F0BDFA0849087818B91A
:1037C00001F081FAFFF740FD00F0CEFA01F0FEFDB6
:1037D0000349012081F8480001BD00000244002097
:1037E000804D00201CB50446E73808280AD26946F7
:1037F0002046FFF787FE0098401C0090694620464F
:10380000FFF7A0FE13BD30B4002513E050F8042BE1
:10381000D30744BFA9F101039A18091F042942F8EC
:10382000045BFAD213468C0744BF15809B1CC90762
:1038300048BF1D7050F8041B0029E7D130BC704709
:10384000DFF834030FF2AD23036100210170C17171
:10385000704738B5DFF820430546207808B100F0FE
:1038600069FA0121C54A2170107818B1BDE83240CB
:103870001D205AE1657028460228C14D02D101F091
:103880006AFE19E000281CBF012800F053FA00204E
:1038900020712A68BB49907D420660784CBF91F840
:1038A000462091F8252020B9C87810B1022AC8BF57
:1038B0000222A27000F03BF8E179B1B9286808B99A
:1038C00000F038FA2868B04D4268117801F0200104
:1038D000A171EE2391786171017A501E8A1C0270E9
:1038E0002B60491CC9B201F0A7F9FFF74DFAA749AF
:1038F0000A78451EA6480078AD41ED0F024307D176
:10390000832020700DB1FFF73BFABDE8314023E082
:10391000202804D10E2104F10800FEF7CFFE02207A
:1039200020701DB1BDE83140FFF72ABA31BD10B596
:10393000FFF790FC904B93F9022001249440611E04
:103940000840D870587818B9BDE8104001F0BDBDE6
:10395000BDE8104001F0A6BD8E488D4A01684908B7
:10396000490001600020107083494878022808BF90
:1039700001F005BE10B5804C607840B9FDF794F9B0
:10398000E178814203D3BDE810401C20CDE0BDE8C2
:10399000104001F0B5BD10B5774C0121E171ED206B
:1039A000FFF720FF6078BDE8104052E780B5774907
:1039B000774B0A781878024318BF00F0BBF9FFF77D
:1039C000E3F96D490A78401E8041C00F022A07D1F1
:1039D00083230B7008B1FFF7D3F9BDE80140BBE7C3
:1039E00018B1BDE80140FFF7CBB901BD10B5624C7D
:1039F000607800281CBF012800F09CF9042020708A
:103A000000F039F921796448491C2171C9B2027862
:103A10008A4203D2BDE81040E12086E0A178407BD5
:103A20004A1C8242B8BF481CA070FFF780FF832069
:103A30002070BDE810409DE710B5FFF7A5F94E498D
:103A4000441EA4410878E40F83280ED1887940B938
:103A500085220A700CB1FFF793F9BDE810400020F1
:103A600063E08620087001F0E9FD04B13DE010BD7F
:103A7000F8B504460D46FFF787F93F4F461EB6419D
:103A80003878F60F862812D18721397001F04AFE66
:103A90000EB1FFF775F97879844204D1002D0CBF7F
:103AA00000201B2000E0E920BDE8F2403DE01EB10F
:103AB000BDE8F140FFF764B9F1BD10B5FFF764F957
:103AC000441E2D480178A441E40F86290AD187229B
:103AD000027001F027FE0CB1FFF752F9BDE810406B
:103AE000E92022E004B100E010BDBDE81040FFF77E
:103AF00047B90000264810B501781F4C20290ED187
:103B000024490A68520852000A6000210170207896
:103B1000022801BF1D4908780028FFF747FF04F17C
:103B20000800BDE81040FEF7E2BD10B5044612489B
:103B300000211B2CC171017004D01848017801F0DC
:103B4000FE01017000F097F8FFF7BFFBFFF7EFFBF6
:103B50002046BDE81040FDF710B910B5084C2068AC
:103B600008B900F0E7F800F036F92168C86000F005
:103B7000C6FE2168088210BD985200200244002031
:103B800040430020804D00203888084084520020A7
:103B90008652002090860840A44D0020F752002055
:103BA0005E48002141700170704738B5050008BFBC
:103BB00000F0C0F8FFF7E8F8441E58484178A441E7
:103BC0000D43457000F070F8E40F1CB1BDE83140C2
:103BD000FFF7D6B831BD10B5040008BF00F0AAF851
:103BE000FFF7D2F84D494A78401E80411443C00F78
:103BF0004C7000B13BE010BD10B5040008BF00F0F0
:103C000099F8FFF7C1F845494A78401E84F0FF044F
:103C100080411440C00F4C7008B1FFF7B1F8BDE807
:103C2000104028E010B5FFF7AFF83C49401E804136
:103C300000224A700A70EF2239490A60ED240C60B4
:103C4000C00F0C6008B1FFF79BF8BDE8104001F011
:103C500044B810B5FFF798F83049441EA44148789D
:103C6000E40F08B100F020F804B100E010BDBDE899
:103C70001040FFF785B810B5FFF786F82749441EB6
:103C8000A4414878E40F60B926490878020608D4B0
:103C90002549087828B925490878020658BF00F058
:103CA00017F804B1E3E710BD80B5FFF76DF81B4AC4
:103CB000411E89411078C90F20B901231370E320F8
:103CC000174A106019B1BDE80140FFF759B801BDAE
:103CD00070B5FFF759F81149451EAD410878ED0F51
:103CE000A8B10022124E0A70EF207060ED217160C1
:103CF0007160FFF749F8441EA4412A20FFF7C8F875
:103D00006FF00400E40F30600CB1FFF739F81DB11B
:103D1000BDE87040FFF734B870BD0000F6520020D7
:103D20003888084084520020865200209852002093
:103D30003488084070470C0080B5002000F023FE56
:103D40004FF47F0000F01AF847486FF00801416017
:103D50006FF01001026842F00802026041600268E0
:103D600042F01002026001BD3F48016821F01001DD
:103D70000160026822F008020260DDE738B50546FE
:103D800000F0D0FDA84228BFFFF7D4FFFEF7FCFFEC
:103D9000441E364805602846A44100F035FEE40F75
:103DA00004B100E031BDBDE83140FEF7E9BF38B5F0
:103DB000FEF7EAFF441EA44100F0B4FDE40F0546FF
:103DC0000CB1FEF7DDFF294801688D4201D30020C8
:103DD00032BD284632BD38B5FEF7D6FF441EA44199
:103DE00000F0B6FDE40F05460CB1FEF7C9FF1F4811
:103DF00001688D4201D3002032BD284632BD70B526
:103E00001A4D04462868844228BFFFF793FFFEF747
:103E1000BBFF6C60461E2046B64100F0D4FD00F0AA
:103E200081FDF60F84420AD111496FF0100008603D
:103E30000EB1FEF7A5FFBDE87040FEF7ADBB1EB1A9
:103E4000BDE87040FEF79CBF70BD7047FEF7A4BB95
:103E500080B500F09FFEBDE80140FEF7EBBB0348D4
:103E600000687047000000000888084008540020DF
